:020000040000FA
:020000000728CF
:020008000900ED
:04000A00003400348A
:02000E0083125B
:1000100085018701073099008316910183128316A9
:10002000871683160F30920083120C3095008312CE
:100030000830930083128C108312920112158312E0
:100040008C1C20288316871283168030910083161B
:1000500070309F0083129D309F0083160712051297
:10006000831207160516AB01AC012C30A30001303A
:10007000A4000530A800C8301A23A80B3B28B422DE
:100080000530A800C8301A23A80B42285030EF22B0
:100090004930EF224330EF225F30EF225330EF221E
:1000A0004F30EF224C30EF224430EF222030EF224D
:1000B0007630EF223130EF222E30EF223130EF2236
:1000C0006430A800C8301A23A80B62288030FA22B6
:1000D0002C188D28051607162D30EF222D30EF2213
:1000E0002D30EF222030EF225330EF224C30EF2220
:1000F0004530EF224530EF225030EF224930EF22D9
:100100004E30EF224730EF222030EF222D30EF2209
:100110002D30EF222D30EF22C92805121E212D0887
:10012000A5002E08A60026082402031D9B282508EA
:1001300023020319A328031CA028FF300712A428B8
:1001400020300716A428DB30EF222508AD00260852
:10015000AE00AF01B0011D2203300621DF30EF22D7
:100160004330EF222030EF222030EF222030EF22E8
:100170002030EF227E30EF222308AD002408AE00AD
:10018000AF01B0011D2203300621DF30EF224330E2
:10019000EF220423AA00031903292B08031D0329B6
:1001A00001302A02031DD7280130AC0603292C1C7C
:1001B000032902302A02031DDE28032904302A0203
:1001C000031DF12800302402031DEA2864302302B5
:1001D00003190329F630A3070318A40AFF30A40764
:1001E000032908302A02031D032901302402031DBC
:1001F000FD28C2302302031903290A30A30703187C
:10020000A40A0030A4072A08AB006628A7003A30E9
:1002100084000A30A80027080A3CA90003191729FE
:100220000008031D1729840AA803A90B1029000838
:10023000303EEF22840AA80B17290800A001A10173
:10024000A2010030A9000A30A80000000000000050
:1002500000000000A80B25299F149F182D29831644
:100260001E088312A007031C3829A10A0319A20A39
:1002700083121E088312A1070318A20AA90B2329BF
:100280002108AD002208AE00AF01B0014130B1003D
:100290008A30B2000D30B3000030B4007521403018
:1002A000B1004230B2000F30B3000030B4008C21F6
:1002B0002830B1000030B2000030B3000030B4008C
:1002C0006821B01F0800AD01AE01AF01B001080008
:1002D0008F220318080030083406C4005822031087
:1002E00034083006C41F803E0800C4017922031C74
:1002F0008C2203180800672274221F30C5009F2239
:10030000380D03185822031C300D03180800C50BC4
:100310007F2944187C220800C401310832043304C8
:100320003404003C031C7922031C8C2203180800AF
:10033000B501B601B701B8019F221F30C5009F2249
:1003400034083802031DAE2933083702031DAE29D5
:1003500032083602031DAE2931083502031CC029BC
:100360003108B5023208031C320FB6023308031CF1
:10037000330FB7023408031C340FB80203102D14D6
:10038000C50B9F2944187C220800C4017922031060
:10039000A32234083802031DD72933083702031D6E
:1003A000AE2932083602031DD72931083502031C55
:1003B000E229AD0FE229AE0FE229AF0FE229B00A20
:1003C0000319080044187C220800300D03180800A7
:1003D000672270221030C500B50DB60DB70DB80DEF
:1003E000B10DB20DB30DB50DB60DB70DB80DB10D04
:1003F000B20DB30D0314AD0DAE0DAF0D2F083302CA
:10040000031D082A2E083202031D082A2D08310276
:10041000031C152A2D08B1022E08031C2E0FB20250
:100420002F08031C2F0FB302AD142D10C50BEC29A0
:100430000310AF0CAE0CAD0C0800C40179220318F8
:100440000800A8222030C500AD0DAE0DAF0DB00DD7
:10045000433084000A30C600800D0A3000020318C1
:1004600080008403C60B2C2AC50B242A4418391497
:1004700003100800C4002030C5003930840044084F
:10048000C6000A300310840A03188007800CC60BCC
:10049000432AB00CAF0CAE0CAD0CC50B3D2A0008C6
:1004A000FF3E031C300D0318080039187C22080099
:1004B0003108AD0732080318320FAE0733080318AE
:1004C000330FAF0734080318340FB00708002D08A6
:1004D000B5002E08B6002F08B7003008B800080095
:1004E000B101B201B301B401AD01AE01AF01B00180
:1004F0000800300D031C080030088039AD09AE0932
:10050000AF09B009AD0F892AAE0F892AAF0F892A2A
:10051000B00AC40A30070800340D031C0800340870
:100520008039B109B209B309B409B10F9C2AB20FDD
:100530009C2AB30F9C2AB40AC40A34070800AD0DE4
:10054000AE0DAF0DB00DB50DB60DB70DB80D080061
:10055000B901BA01BB01BC01BD01BE01BF01C001AF
:08056000C101C201C301080042
:0805680083160511071087102E
:1005700007118510051083128510FA301A233030C8
:10058000E12205140510FA301A2305140510FA307B
:100590001A2305140510FA301A232030E12205141D
:1005A0000510FA301A232030FA22FA301A23C70134
:1005B0000C30FA220130FA220630FA228030FA2278
:1005C00008000711871007100511C900C91B051580
:1005D000491B0714C91A8714491A07150800C800CF
:1005E000E122851405140510480EE12205140510BA
:1005F0001F230800C800E122851005140510480ECD
:10060000E12205140510143083160515071487140C
:10061000071583120301051D0838071C0438871CC1
:100620000238071D013883160511071087100711BE
:1006300083120800CC001F23CC0B1B2B0800313089
:08064000CB00CB0B212B0800BD
:02400E00D433A9
:00000001FF
